:020000040000FA
:0600000000008A15312FFB
:0A1E54008A152A2F8A018A152C2F07
:0E1E6200031E2C2F903098008316181598162A
:101E70001F30990083120330FA00213090000C14B7
:101E80008627EA3A031D582FFA015F2F8627F900AB
:101E9000E33A0319612F7908EA3A03195F2F7908A9
:101EA000ED3A031D462FE43081270330FA008627E0
:101EB000900198018316980183128C012C2FEB302E
:101EC0007F2F8627F6008627F5008627F100FB0086
:101ED0008627F300F2012030840086278000F20775
:101EE000840AFB0B6D2F72087306E830031D7F2FE9
:101EF000E730812798270038E4300319E53081273F
:101F0000462F64000C1E812F9900080064007A0897
:101F10000319942F0C1C942F1010FA0B902F0034DF
:101F20000C100B308F0010148C1E862F1A0808001E
:101F30007508F7007608F800FB010230F40071081C
:101F40007B02031801347B08203E84002130780294
:101F5000031783160319B62F8C1783010F307802ED
:101F60002A30031977020318F82FB82F8C13830136
:101F7000770803178D0003137808031DCD2F043055
:101F800077020318CD2F031783168C1FCA2F8312D5
:101F90002D308D0783010F30CE2F780803178F0067
:101FA00000088E00840A00088C0083160C1555303A
:101FB0008D00AA308D008C140000000083016400A5
:101FC0000D1EDF2F0D12831603170C110C140000C9
:101FD00000008312840300080E06031DF42F840AF8
:101FE00000080C060319F82F8301F40B9F2F00340F
:0E1FF00003130230FB07F70A0319F80A9D2FAE
:084000000200010000000000B5
:02400E00B23FBF
:00000001FF
